:1000000009C00EC00DC00CC00BC00AC009C008C09A
:1000100007C006C011241FBECFE9CDBF5BD0ECC026
:10002000EFCF86E087BB0895813011F4C29A08951E
:10003000882311F4C2980895823021F488B394E0A3
:10004000892788BB089586B1846886B9089564E0DD
:1000500070E0ABD0806287B9369A3699FECF85B111
:1000600090E00895C198E1EEF4E03197F1F700C017
:1000700000004AE050E020E032E0C19AE9EFF0E011
:100080003197F1F700C00000C198B90168237923C6
:100090006115710529F0EDEEF2E03197F1F704C03A
:1000A000E9EFF0E03197F1F700C0000035952795B2
:1000B0004150504011F7C19A89EF90E00197F1F754
:1000C00000C00000C198E1EEF4E03197F1F700C004
:1000D000000008951F9387EA91E60197F1F700C0A9
:1000E000000086E087BB83ED90E30197F1F700C045
:1000F000000081E099DF87EA91E60197F1F700C0FF
:100100000000A1DF87EA91E60197F1F700C0000047
:1001100082E090E09CDF87EA91E60197F1F700C06A
:10012000000083E090E093DF87EA91E60197F1F722
:1001300000C0000080E078DF81E076DF82E090E0C0
:1001400086DF182F91E29A95F1F7000083E090E0A6
:100150007EDF103538F021E030E0163A28F420E058
:1001600030E002C022E030E0803510F4246003C0AB
:10017000863A08F02860B0992061C90175E0880FBF
:10018000991F7A95E1F7822B932B6CDF89E698E132
:100190000197F1F700C0000080E046DF8DE399E4AD
:1001A0000197F1F700C00000C7CF97FB092E072683
:1001B0000AD077FD04D00CD006D000201AF4709538
:1001C00061957F4F0895F6F7909581959F4F08951B
:1001D000AA1BBB1B51E107C0AA1FBB1FA617B7076D
:1001E00010F0A61BB70B881F991F5A95A9F7809589
:0C01F0009095BC01CD010895F894FFCF5C
:00000001FF
